:020000020000FC
:020000005EC0E0
:02009000F5C3B6
:0200A8002EC266
:1000BC0055C101E20EBF0FEF0DBF07E104B908E017
:1000CC0005B901E00DBD00E50CBD289A2C98179AD6
:1000DC000F9A0CE000936A0000E20DBBEE27CC27D0
:1000EC00F2E0D2E0B5E0AA277FEF84E0769A6E9A30
:1000FC0054E016D101E000937E0000EC00937C00EC
:10010C0000E00093A90000E10093A800689A74989D
:10011C0008E90093C9000CE00093CC0063D000EE1A
:10012C0028980BD10FEF09D1289A01EE289805D108
:10013C000AEA03D1289A02EE2898FFD00DECFDD0E4
:10014C00289A03EE2898F9D00BEAF7D0289A08ECF5
:10015C002898F3D006E3F1D0289A05EC2898EDD036
:10016C0000E8EBD0289A0CEE2898E7D008E3E5D00D
:10017C00289A0EEE2898E1D007E0DFD0289A0DEEF1
:10018C002898DBD008EFD9D0289A0FE82898D5D03A
:10019C00289A0FEF0CBB78940000000000000000C0
:1001AC000000000000000000000000000000000043
:1001BC00F3CFFD1303C0EC1301C0EECF2FEF96D19C
:1001CC002191122E93D1219191D11A94E1F72FEF15
:1001DC008DD12AEA8BD12EEF89D12DEF87D1F2FD6B
:1001EC00F2E0DACF02EC2898A8D008E0A6D0289A42
:1001FC0001E82898A2D000E0A0D0289A0830C1F7D6
:10020C00089502EC289899D009E097D0289A01E833
:10021C00289893D000E091D0289A0930C1F708951E
:10022C0002EC28988AD006E188D0289A01E8289810
:10023C0084D000E082D0289A0631C1F7089502ECF0
:10024C0028987BD009E179D0289A01E8289875D0B4
:10025C0000E073D0289A0931C1F7089507E828986F
:10026C006CD000E06AD0902E289A00E2289865D0D5
:10027C0000E063D0065009930350002E00E05DD0DF
:10028C0000E05BD000E059D009930A9501F400E03E
:10029C0054D000E052D000E050D000E04ED000E04E
:1002AC004CD009930A94D9F700E047D000E045D030
:1002BC0000E043D0289A09939992D2FDD2E0089598
:1002CC00B5DF9FDF0FE8289838D000E036D0289AA9
:1002DC0003FDC4DFB4DF2C9A00002C9800E62898AC
:1002EC002CD00D91902F18E0010F27D001E625D0CE
:1002FC0008E823D00D9121D00DEC1FD00BEA1DD0B6
:10030C000D911BD00D9119D00FEF17D00AEA15D013
:10031C00935021F00D9111D09A95E1F7289A0895F8
:10032C004FEF11D0000000000000000000000000A2
:10033C00000000005A95A1F708950EBD0DB507FFFA
:10034C00FDCF0EB508950000000000000000000075
:10035C000000000000004A95B1F708950FB70F9305
:10036C00769A08E00093210100E0009373000F914E
:10037C000FBF189502E82898E0DF00E0DEDF289A2E
:10038C00007E003648F100E22898D7DF00E0D5DF88
:10039C0000E0D3DF08500993102F00E0CEDF00E01F
:1003AC00CCDF00E0CADF099300E0C7DF00E0C5DF67
:1003BC0000E0C3DF099300E0C0DF0993135049F05C
:1003CC0000E0BBDF00E0B9DF00E0B7DF09931A956E
:1003DC00D9F7289AD2FDD2E014DF22DF0F910FBF9C
:1003EC0018950FB70F930FE82898A7DF289A01E804
:1003FC002898A3DF00E0A1DF289A063139F00131FB
:10040C0029F00F31A1F3023191F3B4CF07E828980A
:10041C0094DF00E092DF902E289A00E228988DDF7E
:10042C0000E08BDF06500993102F0350002E00E0E4
:10043C0084DF00E082DF00E080DF09930130D9F037
:10044C0000E07BDF00E079DF00E077DF00E075DFC4
:10045C0000E073DF09930A94D9F700E06EDF00E047
:10046C006CDF00E06ADF289A09939992D2FDD2E002
:10047C000F910FBF189500E060DF00E05EDF00E039
:10048C005CDF00E05ADF00E058DF09930A94D9F7EB
:10049C0000E053DF00E051DF00E04FDF289A0993C2
:1004AC009992C4DEAEDECBDE2C9A00002C982497F9
:1004BC0000E6289842DF0BE040DF01E63EDF08E86B
:1004CC003CDF06E03ADF0DEC38DF0BEA36DF099152
:1004DC0034DF099132DF0FEF30DF0AEA2EDF289A82
:1004EC002296D2FDD2E00F910FBF1895A090C800B4
:1004FC00A5FEFCCF2093CE00089508E00093A10048
:10050C0000E0009372007FEFA0E018950FB70F93F7
:10051C008A9519F00F910FBF189586B4002706BD68
:10052C007BD00FED00937A0084E00F910FBF1895EC
:10053C000FB70F9350907800209079000F910FBF58
:10054C0018955AD13BD1709A0000000070980000A9
:10055C000000709A00000000709800000000709A73
:10056C0000000000709800000000709A000000006D
:10057C00709800000000709A0000000070986C9851
:10058C00000000000000000000000000709A000055
:10059C000000709800000000709A00000000709835
:1005AC006C9A709A0000000070981CD16C9A709A2A
:1005BC0000000000709800000000709A000000001D
:1005CC00709800000000709A000000007098000005
:1005DC000000709A00000000709800000000709AF3
:1005EC0000000000709800000000709A00000000ED
:1005FC00709800000000709A0000000070986C98D1
:10060C00000000000000000000000000709A0000D4
:10061C0000007098E7D00895D1D0709A00000000C7
:10062C00709800000000709A0000000070980000A4
:10063C000000709A00000000709800000000709A92
:10064C0000000000709800000000709A000000008C
:10065C00709800000000709A0000000070986C9870
:10066C00000000000000000000000000709A000074
:10067C000000709800000000709A00000000709854
:10068C00B1D0EC9A08951FB71F9366F0EC9866D022
:10069C005ED0302E63D056D0402E19D01F911FBF84
:1006AC00689418955BD053D059D04CD0C02E07E02D
:1006BC00099303E009935992299249923992C9926C
:1006CC008992D2FDD2E01F911FBFE894189576D085
:1006DC00709A00000000709800000000709A0000F2
:1006EC000000709800000000709A000000007098E4
:1006FC0000000000709A00000000709800000000DC
:10070C00709A0000000070986C98000000000000C7
:10071C00000000000000709A0000000070986C9AB5
:10072C00709A0000000070986C98000000000000A7
:10073C00000000000000709A00000000709852D079
:10074C00EC9A0895709A00000000709808956C9AC5
:10075C00709A0000000070986C9808950027709AA9
:10076C0064990068709800000000709A64990064A5
:10077C00709800000000709A6499006270980000F4
:10078C000000709A64990061709800000000709AE3
:10079C0064990860709800000000709A6499046075
:1007AC00709800000000709A6499026070980000C4
:1007BC000000709A64990160709808956C98709814
:1007CC0000000000709A6C9A709800000000709AFB
:1007DC006C98000000000000000000000000709801
:1007EC006C9A08956C986499FECF709A0000000082
:1007FC007098649BFECF08956C98709A000000006E
:10080C00709800000000709A0000000070980000C2
:10081C000000709A00000000709800000000709AB0
:10082C0000000000709800000000709A00000000AA
:10083C00709800000000709A000000007098000092
:10084C000000709A00000000709800000000709A80
:10085C0000000000709800000000709A000000007A
:10086C00709800000000709A0000000070980895C5
:10087C000FB70F9300E00093A5000093A400009124
:10088C00CE007F3F71F40F3F49F40FE209BB02E049
:10089C00009372000DE00093A10077270F910FBF1A
:1008AC001895772331F4AA270D93702F0F910FBF52
:1008BC0018950D937A9591F7A0E00D91033038F1CE
:1008CC00003428F50D91083011F50D91053BF9F424
:1008DC000D910A3AE1F40D910830C9F40D91073BE2
:1008EC00B1F40D91093B99F476981FEF10932901FF
:1008FC0010E01093280110932501109324011FE29E
:10090C001ABB12E0109373001DE01093210108E054
:10091C000093A10000E0009372007FEF0F910FBFD6
:02092C0018951C
:00000001FF
